C51 COMPILER V9.51   CYFITTER_CFG                                                          10/14/2013 23:29:20 PAGE 1   


C51 COMPILER V9.51, COMPILATION OF MODULE CYFITTER_CFG
OBJECT MODULE PLACED IN .\DP8051\DP8051_Keil_951\Debug\cyfitter_cfg.obj
COMPILER INVOKED BY: C:\Program Files (x86)\Cypress\PSoC Creator\3.0\PSoC Creator\import\keil\pk51\9.51\C51\BIN\c51.exe 
                    -.\Generated_Source\PSoC3\cyfitter_cfg.c NOIV LARGE MODDP2 OMF2 VB(1) PR(.\DP8051\DP8051_Keil_951\Debug\cyfitter_cfg.lst)
                    - CD DB NOIP OT(2,SIZE) INCDIR(.,.\Generated_Source\PSoC3) OJ(.\DP8051\DP8051_Keil_951\Debug\cyfitter_cfg.obj)

line level    source

   1          /*******************************************************************************
   2          * FILENAME: cyfitter_cfg.c
   3          * PSoC Creator 3.0
   4          *
   5          * Description:
   6          * This file is automatically generated by PSoC Creator with device 
   7          * initialization code.  Except for the user defined sections in
   8          * CyClockStartupError(), this file should not be modified.
   9          *
  10          ********************************************************************************
  11          * Copyright 2013, Cypress Semiconductor Corporation.  All rights reserved.
  12          * You may use this file only in accordance with the license, terms, conditions, 
  13          * disclaimers, and limitations in the end user license agreement accompanying 
  14          * the software package with which this file was provided.
  15          ********************************************************************************/
  16          
  17          #include <string.h>
  18          #include <cytypes.h>
  19          #include <cydevice_trm.h>
  20          #include <cyfitter.h>
  21          #include <CyLib.h>
  22          #include <cyfitter_cfg.h>
  23          
  24          #define CY_NEED_CYCLOCKSTARTUPERROR 1
  25          
  26          
  27          #if defined(__C51__) || defined(__CX51__)
  28                  #define CYPACKED
  29                  #define CYPACKED_ATTR
  30                  #define CYALIGNED
  31                  #define DMAINITSEC
  32              #define CY_CFG_UNUSED
  33                  #define CY_CFG_MEMORY_BARRIER() do { } while (0)
  34          
  35          
  36          
  37                  #define CYMEMZERO(a,c) cymemzero((a),(c))
  38                  #define CYCONFIGCPY(d,s,c) cyconfigcpy((c),(s),(d))
  39                  #define CYCONFIGCPYCODE(d,s,c) cyconfigcpycode((c),(s),(d))
  40          #else
                      #error Unsupported toolchain
              #endif
  43          
  44          
  45          
  46          /* Clock startup error codes                                                   */
  47          #define CYCLOCKSTART_NO_ERROR    0u
  48          #define CYCLOCKSTART_XTAL_ERROR  1u
  49          #define CYCLOCKSTART_32KHZ_ERROR 2u
  50          #define CYCLOCKSTART_PLL_ERROR   3u
  51          
  52          #ifdef CY_NEED_CYCLOCKSTARTUPERROR
  53          /*******************************************************************************
C51 COMPILER V9.51   CYFITTER_CFG                                                          10/14/2013 23:29:20 PAGE 2   

  54          * Function Name: CyClockStartupError
  55          ********************************************************************************
  56          * Summary:
  57          *  If an error is encountered during clock configuration (crystal startup error,
  58          *  PLL lock error, etc.), the system will end up here.  Unless reimplemented by
  59          *  the customer, this function will stop in an infinite loop.
  60          *
  61          * Parameters:
  62          *   void
  63          *
  64          * Return:
  65          *   void
  66          *
  67          *******************************************************************************/
  68          CY_CFG_UNUSED
  69          static void CyClockStartupError(uint8 errorCode);
  70          CY_CFG_UNUSED
  71          static void CyClockStartupError(uint8 errorCode)
  72          {
  73   1          /* To remove the compiler warning if errorCode not used.                */
  74   1          errorCode = errorCode;
  75   1      
  76   1          /* `#START CyClockStartupError` */
  77   1      
  78   1          /* If we have a clock startup error (bad MHz crystal, PLL lock, etc.),  */
  79   1          /* we will end up here to allow the customer to implement something to  */
  80   1          /* deal with the clock condition.                                       */
  81   1      
  82   1          /* `#END` */
  83   1      
  84   1          /* If nothing else, stop here since the clocks have not started         */
  85   1          /* correctly.                                                           */
  86   1          while(1) {}
  87   1      }
  88          #endif
  89          
  90          /* IDMUX Address: CYREG_IDMUX_DRQ_CTL0 Size (bytes): 6 */
  91          #define BS_IDMUX_VAL ((const uint8 CYFAR *)0x00080000u)
  92          
  93          /* IOPORT_0 Address: CYDEV_PRTDSI_PRT0_BASE Size (bytes): 7 */
  94          #define BS_IOPORT_0_VAL ((const uint8 CYFAR *)0x00080008u)
  95          
  96          /* UDB_1_5_1_CONFIG Address: CYDEV_UCFG_B0_P0_U1_BASE Size (bytes): 128 */
  97          #define BS_UDB_1_5_1_CONFIG_VAL ((const uint8 CYFAR *)0x00080010u)
  98          
  99          /* UDB_1_4_1_CONFIG Address: CYDEV_UCFG_B0_P1_U0_BASE Size (bytes): 128 */
 100          #define BS_UDB_1_4_1_CONFIG_VAL ((const uint8 CYFAR *)0x00080090u)
 101          
 102          /* UDB_1_4_0_CONFIG Address: CYDEV_UCFG_B0_P1_U1_BASE Size (bytes): 128 */
 103          #define BS_UDB_1_4_0_CONFIG_VAL ((const uint8 CYFAR *)0x00080110u)
 104          
 105          /* UWRK_B0_WRK_STATCTL_BITS Address: CYDEV_UWRK_UWRK8_B0_BASE + 0x00000070u Size (bytes): 32 */
 106          #define BS_UWRK_B0_WRK_STATCTL_BITS_VAL ((const uint8 CYFAR *)0x00080190u)
 107          
 108          /* UCFG_BCTL0 Address: CYREG_BCTL0_MDCLK_EN Size (bytes): 16 */
 109          #define BS_UCFG_BCTL0_VAL ((const uint8 CYFAR *)0x000801B0u)
 110          
 111          /* UDB_2_3_HV_ROUTING Address: CYDEV_UCFG_B0_P2_ROUTE_BASE + 0x00000080u Size (bytes): 128 */
 112          #define BS_UDB_2_3_HV_ROUTING_VAL ((const uint8 CYFAR *)0x000801C0u)
 113          
 114          /* UDBSWITCH_1_4 Address: CYDEV_UCFG_B0_P1_ROUTE_BASE Size (bytes): 128 */
 115          #define BS_UDBSWITCH_1_4_VAL ((const uint8 CYFAR *)0x00080240u)
C51 COMPILER V9.51   CYFITTER_CFG                                                          10/14/2013 23:29:20 PAGE 3   

 116          
 117          /* UDB_2_4_HV_ROUTING Address: CYDEV_UCFG_B0_P1_ROUTE_BASE + 0x00000080u Size (bytes): 128 */
 118          #define BS_UDB_2_4_HV_ROUTING_VAL ((const uint8 CYFAR *)0x000802C0u)
 119          
 120          /* UDBSWITCH_1_5 Address: CYDEV_UCFG_B0_P0_ROUTE_BASE Size (bytes): 128 */
 121          #define BS_UDBSWITCH_1_5_VAL ((const uint8 CYFAR *)0x00080340u)
 122          
 123          /* UDB_2_5_HV_ROUTING Address: CYDEV_UCFG_B0_P0_ROUTE_BASE + 0x00000080u Size (bytes): 128 */
 124          #define BS_UDB_2_5_HV_ROUTING_VAL ((const uint8 CYFAR *)0x000803C0u)
 125          
 126          /* DSI3_3_HV_ROUTING Address: CYDEV_UCFG_DSI2_BASE + 0x00000080u Size (bytes): 128 */
 127          #define BS_DSI3_3_HV_ROUTING_VAL ((const uint8 CYFAR *)0x00080440u)
 128          
 129          /* DSISWITCH_1_4 Address: CYDEV_UCFG_DSI1_BASE Size (bytes): 128 */
 130          #define BS_DSISWITCH_1_4_VAL ((const uint8 CYFAR *)0x000804C0u)
 131          
 132          /* DSI3_4_HV_ROUTING Address: CYDEV_UCFG_DSI1_BASE + 0x00000080u Size (bytes): 128 */
 133          #define BS_DSI3_4_HV_ROUTING_VAL ((const uint8 CYFAR *)0x00080540u)
 134          
 135          /* DSISWITCH_1_5 Address: CYDEV_UCFG_DSI0_BASE Size (bytes): 128 */
 136          #define BS_DSISWITCH_1_5_VAL ((const uint8 CYFAR *)0x000805C0u)
 137          
 138          /* DSI3_5_HV_ROUTING Address: CYDEV_UCFG_DSI0_BASE + 0x00000080u Size (bytes): 128 */
 139          #define BS_DSI3_5_HV_ROUTING_VAL ((const uint8 CYFAR *)0x00080640u)
 140          
 141          /* IOPINS0_0 Address: CYREG_PRT0_DM0 Size (bytes): 8 */
 142          #define BS_IOPINS0_0_VAL ((const uint8 CYFAR *)0x000806C0u)
 143          
 144          /* IOPINS0_2 Address: CYREG_PRT2_DM0 Size (bytes): 8 */
 145          #define BS_IOPINS0_2_VAL ((const uint8 CYFAR *)0x000806C8u)
 146          
 147          
 148          /*******************************************************************************
 149          * Function Name: cfg_dma_init
 150          ********************************************************************************
 151          * Summary:
 152          *  This function is used to copy device configuration data from constant values
 153          *  stored in memory into the proper chip configuration registers using DMA.  It
 154          *  pulls data out of the CFG_TD_LISTs to know exactly how/what to configure.
 155          *
 156          * Parameters:  
 157          *   void
 158          *
 159          * Return:
 160          *   void
 161          *
 162          *******************************************************************************/
 163          static void cfg_dma_init(void);
 164          static void cfg_dma_init(void)
 165          {
 166   1              /* TD structure for big-endian systems. Requires 2-byte endian swap */
 167   1              CYPACKED struct td_t {
 168   1                      uint16 size;
 169   1                      uint8 flags;
 170   1                      uint8 next_td_ptr;
 171   1                      uint16 src;
 172   1                      uint16 dest;
 173   1              } CYPACKED_ATTR;
 174   1      
 175   1              /* PHUB_CH1_CFGMEM_CFG0/1 initialization data */
 176   1              DMAINITSEC static const uint8 CYCODE CH1_ADDR_DATA0[] = { 0x01u, 0x00u, 0x00u, 0x00u, 0x00u, 0x00u, 0x00u
             -, 0x00u };
C51 COMPILER V9.51   CYFITTER_CFG                                                          10/14/2013 23:29:20 PAGE 4   

 177   1      
 178   1              /* PHUB_CH2_CFGMEM_CFG0/1 initialization data */
 179   1              DMAINITSEC static const uint8 CYCODE CH2_ADDR_DATA0[] = { 0x01u, 0x00u, 0x00u, 0x00u, 0x00u, 0x00u, 0x01u
             -, 0x00u };
 180   1      
 181   1              /* PHUB_CH5_CFGMEM_CFG0/1 initialization data */
 182   1              DMAINITSEC static const uint8 CYCODE CH5_ADDR_DATA0[] = { 0x01u, 0x00u, 0x00u, 0x00u, 0x08u, 0x00u, 0x00u
             -, 0x00u };
 183   1      
 184   1              /* PHUB_CH6_CFGMEM_CFG0/1 initialization data */
 185   1              DMAINITSEC static const uint8 CYCODE CH6_ADDR_DATA0[] = { 0x01u, 0x00u, 0x00u, 0x00u, 0x08u, 0x00u, 0x01u
             -, 0x00u };
 186   1      
 187   1              /* Initialization data for each DMA channel's TD registers */
 188   1              DMAINITSEC static const uint8 CYCODE DMA_TD_START_CMD[] = { 0x01u, 0x00u, 0x00u, 0x00u, 0x01u };
 189   1      
 190   1              CYALIGNED static uint32 CYXDATA DMA_ZERO_VAL;
 191   1      
 192   1              /* This table holds all of the initialization data necessary for the DMA
 193   1                 process to transfer data from the source location to the destination. */
 194   1              DMAINITSEC static const struct td_t CYCODE CFG_TD_LIST0[] = {
 195   1                      /* Size, Flags, Next, Source, Destination */
 196   1                      { 8u, 0x23u, 0x02u, (uint16)(uint32)(CH1_ADDR_DATA0), (uint16)(CYREG_PHUB_CFGMEM1_CFG0) },      /* TD 1 */
 197   1                      { 8u, 0x23u, 0x03u, (uint16)(uint32)(CH2_ADDR_DATA0), (uint16)(CYREG_PHUB_CFGMEM2_CFG0) },      /* TD 2 */
 198   1                      { 8u, 0x23u, 0x04u, (uint16)(uint32)(CH5_ADDR_DATA0), (uint16)(CYREG_PHUB_CFGMEM5_CFG0) },      /* TD 3 */
 199   1                      { 8u, 0x23u, 0x05u, (uint16)(uint32)(CH6_ADDR_DATA0), (uint16)(CYREG_PHUB_CFGMEM6_CFG0) },      /* TD 4 */
 200   1                      { 5u, 0x23u, 0x06u, (uint16)(uint32)(DMA_TD_START_CMD), (uint16)(CYREG_PHUB_CH1_BASIC_CFG) },   /* TD 5 */
 201   1                      { 5u, 0x23u, 0x07u, (uint16)(uint32)(DMA_TD_START_CMD), (uint16)(CYREG_PHUB_CH2_BASIC_CFG) },   /* TD 6 */
 202   1                      { 5u, 0x23u, 0x08u, (uint16)(uint32)(DMA_TD_START_CMD), (uint16)(CYREG_PHUB_CH5_BASIC_CFG) },   /* TD 7 */
 203   1                      { 5u, 0x23u, 0xFEu, (uint16)(uint32)(DMA_TD_START_CMD), (uint16)(CYREG_PHUB_CH6_BASIC_CFG) },   /* TD 8 */
 204   1                      { 16u, 0x22u, 0x0Au, (uint16)(uint32)(&DMA_ZERO_VAL), (uint16)(CYREG_PRT1_DR) },        /* TD 9 */
 205   1                      { 64u, 0x22u, 0x0Bu, (uint16)(uint32)(&DMA_ZERO_VAL), (uint16)(CYREG_PRT3_DR) },        /* TD 10 */
 206   1                      { 16u, 0x22u, 0x0Cu, (uint16)(uint32)(&DMA_ZERO_VAL), (uint16)(CYREG_PRT12_DR) },       /* TD 11 */
 207   1                      { 16u, 0x22u, 0xFEu, (uint16)(uint32)(&DMA_ZERO_VAL), (uint16)(CYREG_PRT15_DR) },       /* TD 12 */
 208   1                      { 128u, 0x22u, 0x0Eu, (uint16)(uint32)(&DMA_ZERO_VAL), (uint16)(CYDEV_UCFG_B0_P0_U0_BASE) },    /* TD 13 */
 209   1                      { 384u, 0x22u, 0x0Fu, (uint16)(uint32)(&DMA_ZERO_VAL), (uint16)(CYDEV_UCFG_B0_P2_U0_BASE) },    /* TD 14 */
 210   1                      { 2560u, 0x22u, 0x10u, (uint16)(uint32)(&DMA_ZERO_VAL), (uint16)(CYDEV_UCFG_B0_P3_U0_BASE) },   /* TD 15 *
             -/
 211   1                      { 2048u, 0x22u, 0x11u, (uint16)(uint32)(&DMA_ZERO_VAL), (uint16)(CYDEV_UCFG_B1_P2_U0_BASE) },   /* TD 16 *
             -/
 212   1                      { 128u, 0x22u, 0x12u, (uint16)(uint32)(&DMA_ZERO_VAL), (uint16)(CYDEV_UCFG_DSI2_BASE) },        /* TD 17 */
 213   1                      { 1792u, 0x22u, 0x13u, (uint16)(uint32)(&DMA_ZERO_VAL), (uint16)(CYDEV_UCFG_DSI3_BASE) },       /* TD 18 */
 214   1                      { 512u, 0x22u, 0x14u, (uint16)(uint32)(&DMA_ZERO_VAL), (uint16)(CYDEV_UCFG_DSI12_BASE) },       /* TD 19 */
 215   1                      { 16u, 0x22u, 0xFEu, (uint16)(uint32)(&DMA_ZERO_VAL), (uint16)(CYREG_BCTL1_MDCLK_EN) }, /* TD 20 */
 216   1                      { 7u, 0x23u, 0x16u, (uint16)(uint32)(BS_IOPORT_0_VAL), (uint16)(CYDEV_PRTDSI_PRT0_BASE) },      /* TD 21 */
 217   1                      { 32u, 0x23u, 0xFEu, (uint16)(uint32)(BS_UWRK_B0_WRK_STATCTL_BITS_VAL), (uint16)(CYDEV_UWRK_UWRK8_B0_BAS
             -E + 0x00000070u) },   /* TD 22 */
 218   1                      { 128u, 0x23u, 0x18u, (uint16)(uint32)(BS_UDB_1_5_1_CONFIG_VAL), (uint16)(CYDEV_UCFG_B0_P0_U1_BASE) },  /
             -* TD 23 */
 219   1                      { 128u, 0x23u, 0x19u, (uint16)(uint32)(BS_UDB_1_4_1_CONFIG_VAL), (uint16)(CYDEV_UCFG_B0_P1_U0_BASE) },  /
             -* TD 24 */
 220   1                      { 128u, 0x23u, 0x1Au, (uint16)(uint32)(BS_UDB_1_4_0_CONFIG_VAL), (uint16)(CYDEV_UCFG_B0_P1_U1_BASE) },  /
             -* TD 25 */
 221   1                      { 16u, 0x23u, 0x1Bu, (uint16)(uint32)(BS_UCFG_BCTL0_VAL), (uint16)(CYREG_BCTL0_MDCLK_EN) },     /* TD 26 */
 222   1                      { 128u, 0x23u, 0x1Cu, (uint16)(uint32)(BS_UDB_2_3_HV_ROUTING_VAL), (uint16)(CYDEV_UCFG_B0_P2_ROUTE_BASE 
             -+ 0x00000080u) },     /* TD 27 */
 223   1                      { 128u, 0x23u, 0x1Du, (uint16)(uint32)(BS_UDBSWITCH_1_4_VAL), (uint16)(CYDEV_UCFG_B0_P1_ROUTE_BASE) },  /
             -* TD 28 */
 224   1                      { 128u, 0x23u, 0x1Eu, (uint16)(uint32)(BS_UDB_2_4_HV_ROUTING_VAL), (uint16)(CYDEV_UCFG_B0_P1_ROUTE_BASE 
             -+ 0x00000080u) },     /* TD 29 */
 225   1                      { 128u, 0x23u, 0x1Fu, (uint16)(uint32)(BS_UDBSWITCH_1_5_VAL), (uint16)(CYDEV_UCFG_B0_P0_ROUTE_BASE) },  /
             -* TD 30 */
C51 COMPILER V9.51   CYFITTER_CFG                                                          10/14/2013 23:29:20 PAGE 5   

 226   1                      { 128u, 0x23u, 0x20u, (uint16)(uint32)(BS_UDB_2_5_HV_ROUTING_VAL), (uint16)(CYDEV_UCFG_B0_P0_ROUTE_BASE 
             -+ 0x00000080u) },     /* TD 31 */
 227   1                      { 128u, 0x23u, 0x21u, (uint16)(uint32)(BS_DSI3_3_HV_ROUTING_VAL), (uint16)(CYDEV_UCFG_DSI2_BASE + 0x0000
             -0080u) },        /* TD 32 */
 228   1                      { 128u, 0x23u, 0x22u, (uint16)(uint32)(BS_DSISWITCH_1_4_VAL), (uint16)(CYDEV_UCFG_DSI1_BASE) }, /* TD 33
             - */
 229   1                      { 128u, 0x23u, 0x23u, (uint16)(uint32)(BS_DSI3_4_HV_ROUTING_VAL), (uint16)(CYDEV_UCFG_DSI1_BASE + 0x0000
             -0080u) },        /* TD 34 */
 230   1                      { 128u, 0x23u, 0x24u, (uint16)(uint32)(BS_DSISWITCH_1_5_VAL), (uint16)(CYDEV_UCFG_DSI0_BASE) }, /* TD 35
             - */
 231   1                      { 128u, 0x23u, 0xFEu, (uint16)(uint32)(BS_DSI3_5_HV_ROUTING_VAL), (uint16)(CYDEV_UCFG_DSI0_BASE + 0x0000
             -0080u) },        /* TD 36 */
 232   1              };
 233   1      
 234   1              DMA_ZERO_VAL = 0u;
 235   1              CY_SET_REG8((void CYXDATA *)CYREG_PHUB_CFGMEM0_CFG0, 0x10u);    /* set burstcnt */
 236   1              CY_SET_REG8((void CYXDATA *)CYREG_PHUB_CH0_BASIC_CFG, 0x01u);   /* enable ch0 */
 237   1              CY_SET_REG8((void CYXDATA *)(CYREG_PHUB_CH0_BASIC_STATUS+1u), 0x00u);   /* set first TD to 0 */
 238   1              CY_SET_REG16((void CYXDATA *)CYREG_PHUB_TDMEM0_ORIG_TD0, 36u*8u);       /* transfer size */
 239   1              CY_SET_REG8((void CYXDATA *)(CYREG_PHUB_TDMEM0_ORIG_TD0+2u), 0x01u);    /* set next TD to 1 */
 240   1              CY_SET_REG8((void CYXDATA *)(CYREG_PHUB_TDMEM0_ORIG_TD0+3u), 0xA3u);    /* set TD flags */
 241   1              CY_SET_REG16((void CYXDATA *)CYREG_PHUB_TDMEM0_ORIG_TD1, (uint16)((uint32)CFG_TD_LIST0 & 0x0000FFFFu)); /
             -* set td0's src addr */
 242   1              CY_SET_REG16((void CYXDATA *)(CYREG_PHUB_TDMEM0_ORIG_TD1+2u), CYDEV_PHUB_TDMEM1_BASE);  /* set td0's dst a
             -ddr */
 243   1              CY_SET_REG16((void CYXDATA *)CYREG_PHUB_CFGMEM0_CFG1, (uint16)(CYDEV_FLS_BASE >> 16));  /* set ch0's src h
             -igh addr */
 244   1              CY_SET_REG16((void CYXDATA *)(CYREG_PHUB_CFGMEM0_CFG1+2u), (uint16)(CYDEV_PHUB_TDMEM1_BASE >> 16));     /* se
             -t ch0's dst high addr */
 245   1              CY_SET_REG8((void CYXDATA *)(CYREG_PHUB_CH1_BASIC_STATUS+1u), 0x09u);   /* ch1 first TD: 9 */
 246   1              CY_SET_REG8((void CYXDATA *)(CYREG_PHUB_CH2_BASIC_STATUS+1u), 0x0Du);   /* ch2 first TD: 13 */
 247   1              CY_SET_REG8((void CYXDATA *)(CYREG_PHUB_CH5_BASIC_STATUS+1u), 0x15u);   /* ch5 first TD: 21 */
 248   1              CY_SET_REG8((void CYXDATA *)(CYREG_PHUB_CH6_BASIC_STATUS+1u), 0x17u);   /* ch6 first TD: 23 */
 249   1      
 250   1              CY_CFG_MEMORY_BARRIER();
 251   1              CY_SET_REG8((void CYXDATA *)CYREG_PHUB_CH0_ACTION, 0x01u); /* cpu_req */
 252   1              CY_CFG_MEMORY_BARRIER();
 253   1      
 254   1              /* Wait for all DMA transfers to complete */
 255   1              while(0u != (CY_GET_REG8((void CYXDATA *)CYREG_PHUB_CH0_BASIC_STATUS) & 0x01u)){}
 256   1              while(0u != (CY_GET_REG8((void CYXDATA *)CYREG_PHUB_CH1_BASIC_STATUS) & 0x01u)){}
 257   1              while(0u != (CY_GET_REG8((void CYXDATA *)CYREG_PHUB_CH2_BASIC_STATUS) & 0x01u)){}
 258   1              while(0u != (CY_GET_REG8((void CYXDATA *)CYREG_PHUB_CH5_BASIC_STATUS) & 0x01u)){}
 259   1              while(0u != (CY_GET_REG8((void CYXDATA *)CYREG_PHUB_CH6_BASIC_STATUS) & 0x01u)){}
 260   1      
 261   1      
 262   1              CYCONFIGCPY((void CYFAR *)(CYREG_IDMUX_DRQ_CTL0), (const void CYFAR *)(BS_IDMUX_VAL), 6u);
 263   1      
 264   1      }
 265          /*******************************************************************************
 266          * Function Name: ClockSetup
 267          ********************************************************************************
 268          *
 269          * Summary:
 270          *  Performs the initialization of all of the clocks in the device based on the
 271          *  settings in the Clock tab of the DWR.  This includes enabling the requested
 272          *  clocks and setting the necessary dividers to produce the desired frequency. 
 273          *
 274          * Parameters:
 275          *  void
 276          *
 277          * Return:
C51 COMPILER V9.51   CYFITTER_CFG                                                          10/14/2013 23:29:20 PAGE 6   

 278          *  void
 279          *
 280          *******************************************************************************/
 281          static void ClockSetup(void);
 282          static void ClockSetup(void)
 283          {
 284   1              uint32 timeout;
 285   1              uint8 pllLock;
 286   1      
 287   1      
 288   1              /* Configure Digital Clocks based on settings from Clock DWR */
 289   1              CY_SET_XTND_REG16((void CYFAR *)(CYREG_CLKDIST_DCFG0_CFG0), 0x000Bu);
 290   1              CY_SET_REG8((void CYXDATA *)(CYREG_CLKDIST_DCFG0_CFG0 + 0x2u), 0x18u);
 291   1      
 292   1              /* Configure ILO based on settings from Clock DWR */
 293   1              CY_SET_REG8((void CYXDATA *)(CYREG_SLOWCLK_ILO_CR0), 0x02u);
 294   1              CY_SET_REG8((void CYXDATA *)(CYREG_CLKDIST_CR), 0x08u);
 295   1      
 296   1              /* Configure IMO based on settings from Clock DWR */
 297   1              CY_SET_REG8((void CYXDATA *)(CYREG_FASTCLK_IMO_CR), 0x03u);
 298   1              CY_SET_REG8((void CYXDATA *)(CYREG_IMO_TR1), (CY_GET_XTND_REG8((void CYFAR *)CYREG_FLSHID_CUST_TABLES_IMO
             -_3MHZ)));
 299   1      
 300   1              /* Configure PLL based on settings from Clock DWR */
 301   1              CY_SET_XTND_REG16((void CYFAR *)(CYREG_FASTCLK_PLL_P), 0x0008u);
 302   1              CY_SET_XTND_REG16((void CYFAR *)(CYREG_FASTCLK_PLL_CFG0), 0x1251u);
 303   1              /* Wait up to 250us for the PLL to lock */
 304   1              pllLock = 0u;
 305   1              for (timeout = 250u / 10u; (timeout > 0u) && (pllLock != 0x03u); timeout--)
 306   1              { 
 307   2                      pllLock = 0x03u & ((uint8)((uint8)pllLock << 1) | ((CY_GET_REG8((void CYXDATA *)CYREG_FASTCLK_PLL_SR) & 
             -0x01u) >> 0));
 308   2                      CyDelayCycles(10u * 12u); /* Delay 10us based on 12MHz clock */
 309   2              }
 310   1              /* If we ran out of time the PLL didn't lock so go to the error function */
 311   1              if (timeout == 0u)
 312   1              {
 313   2                      CyClockStartupError(CYCLOCKSTART_PLL_ERROR);
 314   2              }
 315   1      
 316   1              /* Configure Bus/Master Clock based on settings from Clock DWR */
 317   1              CY_SET_XTND_REG16((void CYFAR *)(CYREG_CLKDIST_MSTR0), 0x0100u);
 318   1              CY_SET_REG8((void CYXDATA *)(CYREG_CLKDIST_MSTR0), 0x07u);
 319   1              CY_SET_REG8((void CYXDATA *)(CYREG_CLKDIST_BCFG0), 0x00u);
 320   1              CY_SET_REG8((void CYXDATA *)(CYREG_CLKDIST_BCFG2), 0x48u);
 321   1              CY_SET_REG8((void CYXDATA *)(CYREG_CLKDIST_MSTR0), 0x00u);
 322   1              CY_SET_REG8((void CYXDATA *)(CYREG_CLKDIST_LD), 0x02u);
 323   1      
 324   1              CY_SET_REG8((void CYXDATA *)(CYREG_PM_ACT_CFG2), ((CY_GET_REG8((void CYXDATA *)CYREG_PM_ACT_CFG2) | 0x01u
             -)));
 325   1      }
 326          
 327          
 328          /* Analog API Functions */
 329          
 330          
 331          /*******************************************************************************
 332          * Function Name: AnalogSetDefault
 333          ********************************************************************************
 334          *
 335          * Summary:
 336          *  Sets up the analog portions of the chip to default values based on chip
C51 COMPILER V9.51   CYFITTER_CFG                                                          10/14/2013 23:29:20 PAGE 7   

 337          *  configuration options from the project.
 338          *
 339          * Parameters:
 340          *  void
 341          *
 342          * Return:
 343          *  void
 344          *
 345          *******************************************************************************/
 346          static void AnalogSetDefault(void);
 347          static void AnalogSetDefault(void)
 348          {
 349   1              uint8 bg_xover_inl_trim = CY_GET_XTND_REG8((void CYFAR *)(CYREG_FLSHID_MFG_CFG_BG_XOVER_INL_TRIM + 1u));
 350   1              CY_SET_REG8((void CYXDATA *)(CYREG_BG_DFT0), (bg_xover_inl_trim & 0x07u));
 351   1              CY_SET_REG8((void CYXDATA *)(CYREG_BG_DFT1), ((bg_xover_inl_trim >> 4) & 0x0Fu));
 352   1              CY_SET_REG8((void CYXDATA *)CYREG_PUMP_CR0, 0x44u);
 353   1      }
 354          
 355          
 356          /*******************************************************************************
 357          * Function Name: SetAnalogRoutingPumps
 358          ********************************************************************************
 359          *
 360          * Summary:
 361          * Enables or disables the analog pumps feeding analog routing switches.
 362          * Intended to be called at startup, based on the Vdda system configuration;
 363          * may be called during operation when the user informs us that the Vdda voltage
 364          * crossed the pump threshold.
 365          *
 366          * Parameters:
 367          *  enabled - 1 to enable the pumps, 0 to disable the pumps
 368          *
 369          * Return:
 370          *  void
 371          *
 372          *******************************************************************************/
 373          void SetAnalogRoutingPumps(uint8 enabled)
 374          {
 375   1              uint8 regValue = CY_GET_REG8((void CYXDATA *)CYREG_PUMP_CR0);
 376   1              if (enabled != 0u)
 377   1              {
 378   2                      regValue |= 0x00u;
 379   2              }
 380   1              else
 381   1              {
 382   2                      regValue &= (uint8)~0x00u;
 383   2              }
 384   1              CY_SET_REG8((void CYXDATA *)CYREG_PUMP_CR0, regValue);
 385   1      }
 386          
 387          #define CY_AMUX_UNUSED CYREG_BOOST_SR
 388          
 389          
 390          /*******************************************************************************
 391          * Function Name: cyfitter_cfg
 392          ********************************************************************************
 393          * Summary:
 394          *  This function is called by the start-up code for the selected device. It
 395          *  performs all of the necessary device configuration based on the design
 396          *  settings.  This includes settings from the Design Wide Resources (DWR) such
 397          *  as Clocks and Pins as well as any component configuration that is necessary.
 398          *
C51 COMPILER V9.51   CYFITTER_CFG                                                          10/14/2013 23:29:20 PAGE 8   

 399          * Parameters:  
 400          *   void
 401          *
 402          * Return:
 403          *   void
 404          *
 405          *******************************************************************************/
 406          
 407          void cyfitter_cfg(void)
 408          {
 409   1      
 410   1              /* Set Flash Cycles based on max possible frequency in case a glitch occurs during ClockSetup(). */
 411   1              CY_SET_REG8((void CYXDATA *)(CYREG_CACHE_CR), (((CYDEV_INSTRUCT_CACHE_ENABLED) != 0) ? 0xF1u : 0xC0u));
 412   1              /* Setup clocks based on selections from Clock DWR */
 413   1              ClockSetup();
 414   1              /* Set Flash Cycles based on newly configured 24.00MHz Bus Clock. */
 415   1              CY_SET_REG8((void CYXDATA *)(CYREG_CACHE_CR), (((CYDEV_INSTRUCT_CACHE_ENABLED) != 0) ? 0xB1u : 0x80u));
 416   1              /* Enable/Disable Debug functionality based on settings from System DWR */
 417   1              CY_SET_XTND_REG8((void CYFAR *)CYREG_MLOGIC_DEBUG, (CY_GET_XTND_REG8((void CYFAR *)CYREG_MLOGIC_DEBUG) | 
             -0x05u));
 418   1      
 419   1              {
 420   2                      cfg_dma_init();
 421   2      
 422   2                      /* Perform normal device configuration. Order is not critical for these items. */
 423   2                      CYMEMZERO((void CYFAR *)(CYREG_PHUB_CFGMEM0_CFG0), 4u);
 424   2                      CYMEMZERO((void CYFAR *)(CYREG_PHUB_CFGMEM1_CFG0), 4u);
 425   2      
 426   2                      /* Enable digital routing */
 427   2                      CY_SET_XTND_REG8((void CYFAR *)CYREG_BCTL0_BANK_CTL, CY_GET_XTND_REG8((void CYFAR *)CYREG_BCTL0_BANK_CTL
             -) | 0x02u);
 428   2                      CY_SET_XTND_REG8((void CYFAR *)CYREG_BCTL1_BANK_CTL, CY_GET_XTND_REG8((void CYFAR *)CYREG_BCTL1_BANK_CTL
             -) | 0x02u);
 429   2      
 430   2                      /* Enable UDB array */
 431   2                      CY_SET_REG8((void CYXDATA *)CYREG_PM_ACT_CFG0, CY_GET_REG8((void CYXDATA *)CYREG_PM_ACT_CFG0) | 0x40u);
 432   2                      CY_SET_REG8((void CYXDATA *)CYREG_PM_AVAIL_CR2, CY_GET_REG8((void CYXDATA *)CYREG_PM_AVAIL_CR2) | 0x10u)
             -;
 433   2              }
 434   1      
 435   1              /* Perform second pass device configuration. These items must be configured in specific order after the r
             -egular configuration is done. */
 436   1              CYCONFIGCPY((void CYFAR *)(CYREG_PRT0_DM0), (const void CYFAR *)(BS_IOPINS0_0_VAL), 8u);
 437   1              CYCONFIGCPY((void CYFAR *)(CYREG_PRT2_DM0), (const void CYFAR *)(BS_IOPINS0_2_VAL), 8u);
 438   1      
 439   1              /* Switch Boost to the precision bandgap reference from its internal reference */
 440   1              CY_SET_REG8((void CYXDATA *)CYREG_BOOST_CR2, (CY_GET_REG8((void CYXDATA *)CYREG_BOOST_CR2) | 0x08u));
 441   1              if (CYDEV_CHIP_REV_ACTUAL < 5u)
 442   1              {
 443   2                      CY_SET_REG8((void CYXDATA *)CYREG_PWRSYS_WAKE_TR2, 0x3Au);
 444   2              }
 445   1      
 446   1      
 447   1              /* Perform basic analog initialization to defaults */
 448   1              AnalogSetDefault();
 449   1      
 450   1              /* Configure alternate active mode */
 451   1              CYCONFIGCPY((void CYFAR *)CYDEV_PM_STBY_BASE, (const void CYFAR *)CYDEV_PM_ACT_BASE, 14u);
 452   1              CY_SET_REG8((void CYXDATA *)CYREG_PM_STBY_CFG0, CY_GET_REG8((void CYXDATA *)CYREG_PM_STBY_CFG0) & (uint8)
             -~0x02u);        /* Disable CPU */
 453   1      }
C51 COMPILER V9.51   CYFITTER_CFG                                                          10/14/2013 23:29:20 PAGE 9   

ASSEMBLY LISTING OF GENERATED OBJECT CODE


             ; FUNCTION _CyClockStartupError (BEGIN)
                                           ; SOURCE LINE # 71
0000 900000      R     MOV     DPTR,#errorCode
0003 EF                MOV     A,R7
0004 F0                MOVX    @DPTR,A
                                           ; SOURCE LINE # 72
                                           ; SOURCE LINE # 74
0005 900000      R     MOV     DPTR,#errorCode
0008 E0                MOVX    A,@DPTR
0009 FF                MOV     R7,A
000A 900000      R     MOV     DPTR,#errorCode
000D EF                MOV     A,R7
000E F0                MOVX    @DPTR,A
000F         ?C0001:
                                           ; SOURCE LINE # 86
000F 80FE              SJMP    ?C0001
0011 22                RET     
             ; FUNCTION _CyClockStartupError (END)

             ; FUNCTION cfg_dma_init (BEGIN)
                                           ; SOURCE LINE # 164
                                           ; SOURCE LINE # 165
                                           ; SOURCE LINE # 234
0000 7F00              MOV     R7,#00H
0002 7E00              MOV     R6,#00H
0004 7D00              MOV     R5,#00H
0006 7C00              MOV     R4,#00H
0008 900000      R     MOV     DPTR,#DMA_ZERO_VAL
000B 120000      E     LCALL   ?C?LSTXDATA
                                           ; SOURCE LINE # 235
000E 907600            MOV     DPTR,#07600H
0011 7410              MOV     A,#010H
0013 F0                MOVX    @DPTR,A
                                           ; SOURCE LINE # 236
0014 907010            MOV     DPTR,#07010H
0017 7401              MOV     A,#01H
0019 F0                MOVX    @DPTR,A
                                           ; SOURCE LINE # 237
001A 907019            MOV     DPTR,#07019H
001D E4                CLR     A
001E F0                MOVX    @DPTR,A
                                           ; SOURCE LINE # 238
001F 7B02              MOV     R3,#02H
0021 7A78              MOV     R2,#078H
0023 7900              MOV     R1,#00H
0025 7D20              MOV     R5,#020H
0027 7C01              MOV     R4,#01H
0029 120000      E     LCALL   _cywrite16_nodpx
                                           ; SOURCE LINE # 239
002C 907802            MOV     DPTR,#07802H
002F 7401              MOV     A,#01H
0031 F0                MOVX    @DPTR,A
                                           ; SOURCE LINE # 240
0032 907803            MOV     DPTR,#07803H
0035 74A3              MOV     A,#0A3H
0037 F0                MOVX    @DPTR,A
                                           ; SOURCE LINE # 241
0038 7B02              MOV     R3,#02H
003A 7A78              MOV     R2,#078H
C51 COMPILER V9.51   CYFITTER_CFG                                                          10/14/2013 23:29:20 PAGE 10  

003C 7904              MOV     R1,#04H
003E C003              PUSH    AR3
0040 C002              PUSH    AR2
0042 C001              PUSH    AR1
0044 7BFF              MOV     R3,#0FFH
0046 7A00        R     MOV     R2,#HIGH CFG_TD_LIST0
0048 7900        R     MOV     R1,#LOW CFG_TD_LIST0
004A AF01              MOV     R7,AR1
004C AE02              MOV     R6,AR2
004E AD03              MOV     R5,AR3
0050 7C00              MOV     R4,#00H
0052 EF                MOV     A,R7
0053 54FF              ANL     A,#0FFH
0055 FF                MOV     R7,A
0056 EE                MOV     A,R6
0057 54FF              ANL     A,#0FFH
0059 FE                MOV     R6,A
005A ED                MOV     A,R5
005B 5400              ANL     A,#00H
005D FD                MOV     R5,A
005E EC                MOV     A,R4
005F 5400              ANL     A,#00H
0061 FC                MOV     R4,A
0062 AD07              MOV     R5,AR7
0064 AC06              MOV     R4,AR6
0066 D001              POP     AR1
0068 D002              POP     AR2
006A D003              POP     AR3
006C 120000      E     LCALL   _cywrite16_nodpx
                                           ; SOURCE LINE # 242
006F 7B02              MOV     R3,#02H
0071 7A78              MOV     R2,#078H
0073 7906              MOV     R1,#06H
0075 7D08              MOV     R5,#08H
0077 7C78              MOV     R4,#078H
0079 120000      E     LCALL   _cywrite16_nodpx
                                           ; SOURCE LINE # 243
007C 7B02              MOV     R3,#02H
007E 7A76              MOV     R2,#076H
0080 7904              MOV     R1,#04H
0082 7D10              MOV     R5,#010H
0084 7C00              MOV     R4,#00H
0086 120000      E     LCALL   _cywrite16_nodpx
                                           ; SOURCE LINE # 244
0089 7B02              MOV     R3,#02H
008B 7A76              MOV     R2,#076H
008D 7906              MOV     R1,#06H
008F 7D00              MOV     R5,#00H
0091 7C00              MOV     R4,#00H
0093 120000      E     LCALL   _cywrite16_nodpx
                                           ; SOURCE LINE # 245
0096 907029            MOV     DPTR,#07029H
0099 7409              MOV     A,#09H
009B F0                MOVX    @DPTR,A
                                           ; SOURCE LINE # 246
009C 907039            MOV     DPTR,#07039H
009F 740D              MOV     A,#0DH
00A1 F0                MOVX    @DPTR,A
                                           ; SOURCE LINE # 247
00A2 907069            MOV     DPTR,#07069H
00A5 7415              MOV     A,#015H
00A7 F0                MOVX    @DPTR,A
C51 COMPILER V9.51   CYFITTER_CFG                                                          10/14/2013 23:29:20 PAGE 11  

                                           ; SOURCE LINE # 248
00A8 907079            MOV     DPTR,#07079H
00AB 7417              MOV     A,#017H
00AD F0                MOVX    @DPTR,A
                                           ; SOURCE LINE # 250
                                           ; SOURCE LINE # 251
00AE 907014            MOV     DPTR,#07014H
00B1 7401              MOV     A,#01H
00B3 F0                MOVX    @DPTR,A
                                           ; SOURCE LINE # 252
00B4         ?C0010:
                                           ; SOURCE LINE # 255
00B4 907018            MOV     DPTR,#07018H
00B7 E0                MOVX    A,@DPTR
00B8 FF                MOV     R7,A
00B9 EF                MOV     A,R7
00BA 5401              ANL     A,#01H
00BC FF                MOV     R7,A
00BD 7E00              MOV     R6,#00H
00BF EF                MOV     A,R7
00C0 4E                ORL     A,R6
00C1 70F1              JNZ     ?C0010
00C3         ?C0011:
00C3         ?C0012:
                                           ; SOURCE LINE # 256
00C3 907028            MOV     DPTR,#07028H
00C6 E0                MOVX    A,@DPTR
00C7 FF                MOV     R7,A
00C8 EF                MOV     A,R7
00C9 5401              ANL     A,#01H
00CB FF                MOV     R7,A
00CC 7E00              MOV     R6,#00H
00CE EF                MOV     A,R7
00CF 4E                ORL     A,R6
00D0 70F1              JNZ     ?C0012
00D2         ?C0013:
00D2         ?C0014:
                                           ; SOURCE LINE # 257
00D2 907038            MOV     DPTR,#07038H
00D5 E0                MOVX    A,@DPTR
00D6 FF                MOV     R7,A
00D7 EF                MOV     A,R7
00D8 5401              ANL     A,#01H
00DA FF                MOV     R7,A
00DB 7E00              MOV     R6,#00H
00DD EF                MOV     A,R7
00DE 4E                ORL     A,R6
00DF 70F1              JNZ     ?C0014
00E1         ?C0015:
00E1         ?C0016:
                                           ; SOURCE LINE # 258
00E1 907068            MOV     DPTR,#07068H
00E4 E0                MOVX    A,@DPTR
00E5 FF                MOV     R7,A
00E6 EF                MOV     A,R7
00E7 5401              ANL     A,#01H
00E9 FF                MOV     R7,A
00EA 7E00              MOV     R6,#00H
00EC EF                MOV     A,R7
00ED 4E                ORL     A,R6
00EE 70F1              JNZ     ?C0016
00F0         ?C0017:
C51 COMPILER V9.51   CYFITTER_CFG                                                          10/14/2013 23:29:20 PAGE 12  

00F0         ?C0018:
                                           ; SOURCE LINE # 259
00F0 907078            MOV     DPTR,#07078H
00F3 E0                MOVX    A,@DPTR
00F4 FF                MOV     R7,A
00F5 EF                MOV     A,R7
00F6 5401              ANL     A,#01H
00F8 FF                MOV     R7,A
00F9 7E00              MOV     R6,#00H
00FB EF                MOV     A,R7
00FC 4E                ORL     A,R6
00FD 70F1              JNZ     ?C0018
00FF         ?C0019:
                                           ; SOURCE LINE # 262
00FF 7B08              MOV     R3,#08H
0101 7A00              MOV     R2,#00H
0103 7900              MOV     R1,#00H
0105 C003              PUSH    AR3
0107 C002              PUSH    AR2
0109 C001              PUSH    AR1
010B 7B01              MOV     R3,#01H
010D 7A51              MOV     R2,#051H
010F 7910              MOV     R1,#010H
0111 900000      E     MOV     DPTR,#?_cyconfigcpy?BYTE+05H
0114 120000      E     LCALL   ?C?PSTXDATA
0117 D001              POP     AR1
0119 D002              POP     AR2
011B D003              POP     AR3
011D 7F06              MOV     R7,#06H
011F 7E00              MOV     R6,#00H
0121 120000      E     LCALL   _cyconfigcpy
                                           ; SOURCE LINE # 264
0124 22                RET     
             ; FUNCTION cfg_dma_init (END)

             ; FUNCTION ClockSetup (BEGIN)
                                           ; SOURCE LINE # 282
                                           ; SOURCE LINE # 283
                                           ; SOURCE LINE # 289
0000 7B00              MOV     R3,#00H
0002 7A40              MOV     R2,#040H
0004 7980              MOV     R1,#080H
0006 7D0B              MOV     R5,#0BH
0008 7C00              MOV     R4,#00H
000A 120000      E     LCALL   _cywrite16
                                           ; SOURCE LINE # 290
000D 904082            MOV     DPTR,#04082H
0010 7418              MOV     A,#018H
0012 F0                MOVX    @DPTR,A
                                           ; SOURCE LINE # 293
0013 904300            MOV     DPTR,#04300H
0016 7402              MOV     A,#02H
0018 F0                MOVX    @DPTR,A
                                           ; SOURCE LINE # 294
0019 904000            MOV     DPTR,#04000H
001C 7408              MOV     A,#08H
001E F0                MOVX    @DPTR,A
                                           ; SOURCE LINE # 297
001F 904200            MOV     DPTR,#04200H
0022 7403              MOV     A,#03H
0024 F0                MOVX    @DPTR,A
                                           ; SOURCE LINE # 298
C51 COMPILER V9.51   CYFITTER_CFG                                                          10/14/2013 23:29:20 PAGE 13  

0025 7B0C              MOV     R3,#0CH
0027 7A01              MOV     R2,#01H
0029 7908              MOV     R1,#08H
002B 120000      E     LCALL   _cyread8
002E 9046A1            MOV     DPTR,#046A1H
0031 EF                MOV     A,R7
0032 F0                MOVX    @DPTR,A
                                           ; SOURCE LINE # 301
0033 7B00              MOV     R3,#00H
0035 7A42              MOV     R2,#042H
0037 7922              MOV     R1,#022H
0039 7D08              MOV     R5,#08H
003B 7C00              MOV     R4,#00H
003D 120000      E     LCALL   _cywrite16
                                           ; SOURCE LINE # 302
0040 7B00              MOV     R3,#00H
0042 7A42              MOV     R2,#042H
0044 7920              MOV     R1,#020H
0046 7D51              MOV     R5,#051H
0048 7C12              MOV     R4,#012H
004A 120000      E     LCALL   _cywrite16
                                           ; SOURCE LINE # 304
004D 900000      R     MOV     DPTR,#pllLock
0050 E4                CLR     A
0051 F0                MOVX    @DPTR,A
                                           ; SOURCE LINE # 305
0052 7F19              MOV     R7,#019H
0054 7E00              MOV     R6,#00H
0056 7D00              MOV     R5,#00H
0058 7C00              MOV     R4,#00H
005A 900000      R     MOV     DPTR,#timeout
005D 120000      E     LCALL   ?C?LSTXDATA
0060         ?C0021:
0060 900000      R     MOV     DPTR,#timeout
0063 120000      E     LCALL   ?C?LLDXDATA
0066 D3                SETB    C
0067 EF                MOV     A,R7
0068 9400              SUBB    A,#00H
006A EE                MOV     A,R6
006B 9400              SUBB    A,#00H
006D 404E              JC      ?C0022
006F 900000      R     MOV     DPTR,#pllLock
0072 E0                MOVX    A,@DPTR
0073 FF                MOV     R7,A
0074 EF                MOV     A,R7
0075 6403              XRL     A,#03H
0077 6044              JZ      ?C0022
                                           ; SOURCE LINE # 306
                                           ; SOURCE LINE # 307
0079 904225            MOV     DPTR,#04225H
007C E0                MOVX    A,@DPTR
007D FF                MOV     R7,A
007E EF                MOV     A,R7
007F 5401              ANL     A,#01H
0081 FF                MOV     R7,A
0082 7E00              MOV     R6,#00H
0084 900000      R     MOV     DPTR,#pllLock
0087 E0                MOVX    A,@DPTR
0088 FE                MOV     R6,A
0089 EE                MOV     A,R6
008A 25E0              ADD     A,ACC
008C FE                MOV     R6,A
C51 COMPILER V9.51   CYFITTER_CFG                                                          10/14/2013 23:29:20 PAGE 14  

008D EE                MOV     A,R6
008E 4F                ORL     A,R7
008F FF                MOV     R7,A
0090 EF                MOV     A,R7
0091 5403              ANL     A,#03H
0093 FF                MOV     R7,A
0094 900000      R     MOV     DPTR,#pllLock
0097 EF                MOV     A,R7
0098 F0                MOVX    @DPTR,A
                                           ; SOURCE LINE # 308
0099 7F78              MOV     R7,#078H
009B 7E00              MOV     R6,#00H
009D 7D00              MOV     R5,#00H
009F 7C00              MOV     R4,#00H
00A1 120000      E     LCALL   _CyDelayCycles
                                           ; SOURCE LINE # 309
00A4 900000      R     MOV     DPTR,#timeout
00A7 120000      E     LCALL   ?C?LLDXDATA
00AA 7BFF              MOV     R3,#0FFH
00AC 7AFF              MOV     R2,#0FFH
00AE 79FF              MOV     R1,#0FFH
00B0 78FF              MOV     R0,#0FFH
00B2 120000      E     LCALL   ?C?LADD
00B5 900000      R     MOV     DPTR,#timeout
00B8 120000      E     LCALL   ?C?LSTXDATA
00BB 80A3              SJMP    ?C0021
00BD         ?C0022:
                                           ; SOURCE LINE # 311
00BD 900000      R     MOV     DPTR,#timeout
00C0 120000      E     LCALL   ?C?LLDXDATA
00C3 EF                MOV     A,R7
00C4 4E                ORL     A,R6
00C5 7005              JNZ     ?C0024
                                           ; SOURCE LINE # 312
                                           ; SOURCE LINE # 313
00C7 7F03              MOV     R7,#03H
00C9 120000      R     LCALL   _CyClockStartupError
                                           ; SOURCE LINE # 314
00CC         ?C0024:
                                           ; SOURCE LINE # 317
00CC 7B00              MOV     R3,#00H
00CE 7A40              MOV     R2,#040H
00D0 7904              MOV     R1,#04H
00D2 7D00              MOV     R5,#00H
00D4 7C01              MOV     R4,#01H
00D6 120000      E     LCALL   _cywrite16
                                           ; SOURCE LINE # 318
00D9 904004            MOV     DPTR,#04004H
00DC 7407              MOV     A,#07H
00DE F0                MOVX    @DPTR,A
                                           ; SOURCE LINE # 319
00DF 904006            MOV     DPTR,#04006H
00E2 E4                CLR     A
00E3 F0                MOVX    @DPTR,A
                                           ; SOURCE LINE # 320
00E4 904008            MOV     DPTR,#04008H
00E7 7448              MOV     A,#048H
00E9 F0                MOVX    @DPTR,A
                                           ; SOURCE LINE # 321
00EA 904004            MOV     DPTR,#04004H
00ED E4                CLR     A
00EE F0                MOVX    @DPTR,A
C51 COMPILER V9.51   CYFITTER_CFG                                                          10/14/2013 23:29:20 PAGE 15  

                                           ; SOURCE LINE # 322
00EF 904001            MOV     DPTR,#04001H
00F2 7402              MOV     A,#02H
00F4 F0                MOVX    @DPTR,A
                                           ; SOURCE LINE # 324
00F5 9043A2            MOV     DPTR,#043A2H
00F8 E0                MOVX    A,@DPTR
00F9 FF                MOV     R7,A
00FA EF                MOV     A,R7
00FB 4401              ORL     A,#01H
00FD FF                MOV     R7,A
00FE 9043A2            MOV     DPTR,#043A2H
0101 EF                MOV     A,R7
0102 F0                MOVX    @DPTR,A
                                           ; SOURCE LINE # 325
0103 22                RET     
             ; FUNCTION ClockSetup (END)

             ; FUNCTION AnalogSetDefault (BEGIN)
                                           ; SOURCE LINE # 347
                                           ; SOURCE LINE # 348
                                           ; SOURCE LINE # 349
0000 7B0C              MOV     R3,#0CH
0002 7A01              MOV     R2,#01H
0004 79CF              MOV     R1,#0CFH
0006 120000      E     LCALL   _cyread8
0009 900000      R     MOV     DPTR,#bg_xover_inl_trim
000C EF                MOV     A,R7
000D F0                MOVX    @DPTR,A
                                           ; SOURCE LINE # 350
000E 900000      R     MOV     DPTR,#bg_xover_inl_trim
0011 E0                MOVX    A,@DPTR
0012 FF                MOV     R7,A
0013 EF                MOV     A,R7
0014 5407              ANL     A,#07H
0016 FF                MOV     R7,A
0017 90586E            MOV     DPTR,#0586EH
001A EF                MOV     A,R7
001B F0                MOVX    @DPTR,A
                                           ; SOURCE LINE # 351
001C 900000      R     MOV     DPTR,#bg_xover_inl_trim
001F E0                MOVX    A,@DPTR
0020 FF                MOV     R7,A
0021 EF                MOV     A,R7
0022 C4                SWAP    A
0023 540F              ANL     A,#0FH
0025 FF                MOV     R7,A
0026 EF                MOV     A,R7
0027 540F              ANL     A,#0FH
0029 FF                MOV     R7,A
002A 90586F            MOV     DPTR,#0586FH
002D EF                MOV     A,R7
002E F0                MOVX    @DPTR,A
                                           ; SOURCE LINE # 352
002F 905876            MOV     DPTR,#05876H
0032 7444              MOV     A,#044H
0034 F0                MOVX    @DPTR,A
                                           ; SOURCE LINE # 353
0035 22                RET     
             ; FUNCTION AnalogSetDefault (END)

             ; FUNCTION _SetAnalogRoutingPumps (BEGIN)
C51 COMPILER V9.51   CYFITTER_CFG                                                          10/14/2013 23:29:20 PAGE 16  

                                           ; SOURCE LINE # 373
0000 900000      R     MOV     DPTR,#enabled
0003 EF                MOV     A,R7
0004 F0                MOVX    @DPTR,A
                                           ; SOURCE LINE # 374
                                           ; SOURCE LINE # 375
0005 905876            MOV     DPTR,#05876H
0008 E0                MOVX    A,@DPTR
0009 FF                MOV     R7,A
000A 900000      R     MOV     DPTR,#regValue
000D EF                MOV     A,R7
000E F0                MOVX    @DPTR,A
                                           ; SOURCE LINE # 376
000F 900000      R     MOV     DPTR,#enabled
0012 E0                MOVX    A,@DPTR
0013 FF                MOV     R7,A
0014 EF                MOV     A,R7
0015 6010              JZ      ?C0027
                                           ; SOURCE LINE # 377
                                           ; SOURCE LINE # 378
0017 900000      R     MOV     DPTR,#regValue
001A E0                MOVX    A,@DPTR
001B FF                MOV     R7,A
001C EF                MOV     A,R7
001D 4400              ORL     A,#00H
001F FF                MOV     R7,A
0020 900000      R     MOV     DPTR,#regValue
0023 EF                MOV     A,R7
0024 F0                MOVX    @DPTR,A
                                           ; SOURCE LINE # 379
0025 800E              SJMP    ?C0028
0027         ?C0027:
                                           ; SOURCE LINE # 381
                                           ; SOURCE LINE # 382
0027 900000      R     MOV     DPTR,#regValue
002A E0                MOVX    A,@DPTR
002B FF                MOV     R7,A
002C EF                MOV     A,R7
002D 54FF              ANL     A,#0FFH
002F FF                MOV     R7,A
0030 900000      R     MOV     DPTR,#regValue
0033 EF                MOV     A,R7
0034 F0                MOVX    @DPTR,A
                                           ; SOURCE LINE # 383
0035         ?C0028:
                                           ; SOURCE LINE # 384
0035 900000      R     MOV     DPTR,#regValue
0038 E0                MOVX    A,@DPTR
0039 FF                MOV     R7,A
003A 905876            MOV     DPTR,#05876H
003D EF                MOV     A,R7
003E F0                MOVX    @DPTR,A
                                           ; SOURCE LINE # 385
003F 22                RET     
             ; FUNCTION _SetAnalogRoutingPumps (END)

             ; FUNCTION cyfitter_cfg (BEGIN)
                                           ; SOURCE LINE # 407
                                           ; SOURCE LINE # 408
                                           ; SOURCE LINE # 411
0000 904800            MOV     DPTR,#04800H
0003 74F1              MOV     A,#0F1H
C51 COMPILER V9.51   CYFITTER_CFG                                                          10/14/2013 23:29:20 PAGE 17  

0005 F0                MOVX    @DPTR,A
                                           ; SOURCE LINE # 413
0006 120000      R     LCALL   ClockSetup
                                           ; SOURCE LINE # 415
0009 904800            MOV     DPTR,#04800H
000C 74B1              MOV     A,#0B1H
000E F0                MOVX    @DPTR,A
                                           ; SOURCE LINE # 417
000F 7B00              MOV     R3,#00H
0011 7A46              MOV     R2,#046H
0013 79E8              MOV     R1,#0E8H
0015 120000      E     LCALL   _cyread8
0018 EF                MOV     A,R7
0019 4405              ORL     A,#05H
001B FD                MOV     R5,A
001C 7B00              MOV     R3,#00H
001E 7A46              MOV     R2,#046H
0020 79E8              MOV     R1,#0E8H
0022 120000      E     LCALL   _cywrite8
                                           ; SOURCE LINE # 419
                                           ; SOURCE LINE # 420
0025 120000      R     LCALL   cfg_dma_init
                                           ; SOURCE LINE # 423
0028 7B00              MOV     R3,#00H
002A 7A76              MOV     R2,#076H
002C 7900              MOV     R1,#00H
002E 7D04              MOV     R5,#04H
0030 7C00              MOV     R4,#00H
0032 120000      E     LCALL   _cymemzero
                                           ; SOURCE LINE # 424
0035 7B00              MOV     R3,#00H
0037 7A76              MOV     R2,#076H
0039 7908              MOV     R1,#08H
003B 7D04              MOV     R5,#04H
003D 7C00              MOV     R4,#00H
003F 120000      E     LCALL   _cymemzero
                                           ; SOURCE LINE # 427
0042 7B01              MOV     R3,#01H
0044 7A50              MOV     R2,#050H
0046 7903              MOV     R1,#03H
0048 120000      E     LCALL   _cyread8
004B EF                MOV     A,R7
004C 4402              ORL     A,#02H
004E FD                MOV     R5,A
004F 7B01              MOV     R3,#01H
0051 7A50              MOV     R2,#050H
0053 7903              MOV     R1,#03H
0055 120000      E     LCALL   _cywrite8
                                           ; SOURCE LINE # 428
0058 7B01              MOV     R3,#01H
005A 7A50              MOV     R2,#050H
005C 7913              MOV     R1,#013H
005E 120000      E     LCALL   _cyread8
0061 EF                MOV     A,R7
0062 4402              ORL     A,#02H
0064 FD                MOV     R5,A
0065 7B01              MOV     R3,#01H
0067 7A50              MOV     R2,#050H
0069 7913              MOV     R1,#013H
006B 120000      E     LCALL   _cywrite8
                                           ; SOURCE LINE # 431
006E 9043A0            MOV     DPTR,#043A0H
C51 COMPILER V9.51   CYFITTER_CFG                                                          10/14/2013 23:29:20 PAGE 18  

0071 E0                MOVX    A,@DPTR
0072 FF                MOV     R7,A
0073 EF                MOV     A,R7
0074 4440              ORL     A,#040H
0076 FF                MOV     R7,A
0077 9043A0            MOV     DPTR,#043A0H
007A EF                MOV     A,R7
007B F0                MOVX    @DPTR,A
                                           ; SOURCE LINE # 432
007C 9043C2            MOV     DPTR,#043C2H
007F E0                MOVX    A,@DPTR
0080 FF                MOV     R7,A
0081 EF                MOV     A,R7
0082 4410              ORL     A,#010H
0084 FF                MOV     R7,A
0085 9043C2            MOV     DPTR,#043C2H
0088 EF                MOV     A,R7
0089 F0                MOVX    @DPTR,A
                                           ; SOURCE LINE # 433
                                           ; SOURCE LINE # 436
008A 7B08              MOV     R3,#08H
008C 7A06              MOV     R2,#06H
008E 79C0              MOV     R1,#0C0H
0090 C003              PUSH    AR3
0092 C002              PUSH    AR2
0094 C001              PUSH    AR1
0096 7B00              MOV     R3,#00H
0098 7A51              MOV     R2,#051H
009A 7902              MOV     R1,#02H
009C 900000      E     MOV     DPTR,#?_cyconfigcpy?BYTE+05H
009F 120000      E     LCALL   ?C?PSTXDATA
00A2 D001              POP     AR1
00A4 D002              POP     AR2
00A6 D003              POP     AR3
00A8 7F08              MOV     R7,#08H
00AA 7E00              MOV     R6,#00H
00AC 120000      E     LCALL   _cyconfigcpy
                                           ; SOURCE LINE # 437
00AF 7B08              MOV     R3,#08H
00B1 7A06              MOV     R2,#06H
00B3 79C8              MOV     R1,#0C8H
00B5 C003              PUSH    AR3
00B7 C002              PUSH    AR2
00B9 C001              PUSH    AR1
00BB 7B00              MOV     R3,#00H
00BD 7A51              MOV     R2,#051H
00BF 7922              MOV     R1,#022H
00C1 900000      E     MOV     DPTR,#?_cyconfigcpy?BYTE+05H
00C4 120000      E     LCALL   ?C?PSTXDATA
00C7 D001              POP     AR1
00C9 D002              POP     AR2
00CB D003              POP     AR3
00CD 7F08              MOV     R7,#08H
00CF 7E00              MOV     R6,#00H
00D1 120000      E     LCALL   _cyconfigcpy
                                           ; SOURCE LINE # 440
00D4 904322            MOV     DPTR,#04322H
00D7 E0                MOVX    A,@DPTR
00D8 FF                MOV     R7,A
00D9 EF                MOV     A,R7
00DA 4408              ORL     A,#08H
00DC FF                MOV     R7,A
C51 COMPILER V9.51   CYFITTER_CFG                                                          10/14/2013 23:29:20 PAGE 19  

00DD 904322            MOV     DPTR,#04322H
00E0 EF                MOV     A,R7
00E1 F0                MOVX    @DPTR,A
                                           ; SOURCE LINE # 441
00E2 9046EC            MOV     DPTR,#046ECH
00E5 E0                MOVX    A,@DPTR
00E6 FF                MOV     R7,A
00E7 EF                MOV     A,R7
00E8 C3                CLR     C
00E9 9405              SUBB    A,#05H
00EB 5006              JNC     ?C0030
                                           ; SOURCE LINE # 442
                                           ; SOURCE LINE # 443
00ED 904689            MOV     DPTR,#04689H
00F0 743A              MOV     A,#03AH
00F2 F0                MOVX    @DPTR,A
                                           ; SOURCE LINE # 444
00F3         ?C0030:
                                           ; SOURCE LINE # 448
00F3 120000      R     LCALL   AnalogSetDefault
                                           ; SOURCE LINE # 451
00F6 7B00              MOV     R3,#00H
00F8 7A43              MOV     R2,#043H
00FA 79A0              MOV     R1,#0A0H
00FC C003              PUSH    AR3
00FE C002              PUSH    AR2
0100 C001              PUSH    AR1
0102 7B00              MOV     R3,#00H
0104 7A43              MOV     R2,#043H
0106 79B0              MOV     R1,#0B0H
0108 900000      E     MOV     DPTR,#?_cyconfigcpy?BYTE+05H
010B 120000      E     LCALL   ?C?PSTXDATA
010E D001              POP     AR1
0110 D002              POP     AR2
0112 D003              POP     AR3
0114 7F0E              MOV     R7,#0EH
0116 7E00              MOV     R6,#00H
0118 120000      E     LCALL   _cyconfigcpy
                                           ; SOURCE LINE # 452
011B 9043B0            MOV     DPTR,#043B0H
011E E0                MOVX    A,@DPTR
011F FF                MOV     R7,A
0120 EF                MOV     A,R7
0121 54FD              ANL     A,#0FDH
0123 FF                MOV     R7,A
0124 EF                MOV     A,R7
0125 F0                MOVX    @DPTR,A
                                           ; SOURCE LINE # 453
0126 22                RET     
             ; FUNCTION cyfitter_cfg (END)



MODULE INFORMATION:   STATIC OVERLAYABLE
   CODE SIZE        =    984    ----
   CONSTANT SIZE    =    325    ----
   XDATA SIZE       =      4       9
   PDATA SIZE       =   ----    ----
   DATA SIZE        =   ----    ----
   IDATA SIZE       =   ----    ----
   BIT SIZE         =   ----    ----
   EDATA SIZE       =   ----    ----
C51 COMPILER V9.51   CYFITTER_CFG                                                          10/14/2013 23:29:20 PAGE 20  

   HDATA SIZE       =   ----    ----
   XDATA CONST SIZE =   ----    ----
   FAR CONST SIZE   =   ----    ----
END OF MODULE INFORMATION.


C51 COMPILATION COMPLETE.  0 WARNING(S),  0 ERROR(S)
